:020000020000FC
:100000000FE50DBF04E00EBF0FEF07BB00E004BB20
:100010000FEF05BB40E003B383B30E6F0E3F31F02B
:100020008D6F8D3F49F020D015D0F5CF493051F07C
:1000300043951AD00FD0EFCF403041F04A9514D0FD
:1000400009D0E9CF40E010D005D0E5CF49E00CD091
:1000500001D0E1CF30E52FEF1FEF1A95F1F72A9588
:10006000D9F73A95C1F70895403099F04130A1F0A1
:100070004230A9F04330B1F04430B9F04530C1F01E
:100080004630C9F04730D1F04830D9F04930E1F07E
:1000900008950FE308BB089506E008BB08950BE53B
:1000A00008BB08950FE408BB089506E608BB089551
:1000B0000DE608BB08950DE708BB089507E008BBEF
:0E00C00008950FE708BB08950FE608BB0895EA
:00000001FF
